:100000008316640088018030810000308B000F303F
:100010008500C7308600831299019C019A018901ED
:10002000632096009A07632097009A076320980040
:100030009A072D211D08031D21280D301E02031CC7
:10004000292804301D020318292863201A020319E5
:100050002F28643096007D30980097019C14061874
:100060005D28190803193E2119081F390319692051
:1000700019080339031933210C308E0006185D2846
:10008000FA2103194521F62103194021F82103190A
:100090004221EE2103199920F02103199320F22126
:1000A0000319FB20F4210319F120E521FC21031D94
:1000B00040288E0B3E28990A3128692010308B0089
:1000C0006300000000288316081483120808890AB8
:1000D00008009C1C08009C109A01890116087A20CF
:1000E00017087A2018087A201A087A20C0210800F8
:1000F000C021782888009A07831608155530890092
:10010000AA308900881488188328081E85280812B8
:100110000811831208088316081483120802031DAD
:100120007828890A0800FA3016020318EF281C15EF
:100130009F2832301602031CEF280319EF2848309D
:10014000A200E830A1000130A00016085E22323083
:100150001C19B128A207031CB828A10FB828A00AAF
:10016000B828A2020318B8280130A102031CA0037A
:100170002208A4002108A3004830A200E830A10012
:100180000130A0003E2221080319CA28A101FC3039
:10019000A200D028323022020318D0283230A20028
:1001A0001808A4001708A3001608292222089600A0
:1001B0001F08A2001E08A1001D08A00016085E224C
:1001C0002208980021089700160C2602031CEB2831
:1001D000980FEB28970A9C1485211C110800C02158
:1001E000ED282D211D08031DF9280D301E02031CCA
:1001F000EF281C1500292D2103301D020318EF28BC
:100200002D211F08A2001E08A1001D08A000143007
:100210005E221C1916291F08A2071E0803181E0FAC
:10022000A1071D0803181D0FA007262922089F02F9
:100230002108031C210F9E022008031C200F9D0291
:100240001F08A2001E08A1001D08A00016085E22BB
:100250002208980021089700EB281808A400170826
:10026000A3001608292A861B08008615E521E5212A
:10027000E521E521E521732186110800061B080010
:100280008D01472950308D004729A1308D008615FA
:10029000E521E521E521E521E52103308A000D086E
:1002A00000238A018C0000300C02031D592986119D
:1002B000080001300C02031D62298A218A218A214B
:1002C0008A216E2903108C0D031868298021692961
:1002D00079218A2180300C02031D62298A218A211A
:1002E0008A218D0A4D29940195018F218F21962114
:1002F0000800940195018F218F218F2196210800FC
:10030000940195018F2196210800940195018F2178
:1003100099210800940195018F219821080018085F
:10032000950717080318940F9407080006169929D3
:100330001C1405128612AE290000910B9C29061A86
:1003400086161C1C051616089100910391030000E7
:1003500000000000910BA9290512861216089100D1
:1003600091039103910301300000000095020318EE
:100370009C299103940203189C2906121C10080062
:10038000FA3090008F0005120F0891000000000065
:100390000000910BC82905160F089100000000000D
:1003A0000000910BD02905120A308F0296300F02FF
:1003B0000318E2298F0BDA298F0BDC298F0BDE293A
:1003C000FA308F00900BC42908008330900091010F
:1003D000910BE8290000900BE82908000130092A58
:1003E0000230092A0430092A0830092A0230192A61
:1003F0000430192A0630192A0F309B0005081B0506
:100400001B060319080006309B0006081B051B0687
:1004100008009B000A309000910105081B051B068F
:100420001B02031D0800910B0D2A900B0D2A0315CA
:1004300008009B000A309000910106081B051B066E
:100440001B02031D0800910B1D2A900B1D2A03158A
:1004500008009D019E019F000830A70003109F0C1B
:10046000031C382A24089E0723080318230F9D071E
:100470009D0C9E0C9F0CA70B302A0800A501A6011D
:100480001830A700A20DA10DA00DA60DA50DA70D5A
:100490002408A6022308031C230F2502031827148F
:1004A0002718552A2408A6072508A5000310A70C1D
:1004B000A70B422AA20DA10DA00D0800A400A301C4
:0204C0003E2AD2
:10060000820718340134183401341834013420348A
:10061000B0347C340834D0342034943488340134F9
:100620002034B0347C340834D034203494348834CA
:1006300001347834A0340C3404342034B034003421
:1006A20018340134183401342034B0347C34083422
:1006B200D03420349434883401342034B0347C343F
:0C06C2000834D0342034943488340034E0
:1007440018340134183401342034B0347C3408347F
:10075400D034203401342034B0347C340834D034E0
:06076400203401340034D2
:02400E00F13F80
:00000001FF
